S123C0002A204166666963686575724C4344202A002A2020742065207320742E2E2E2020D4
S123C0202A12151515151512008640B710398E00FFBDC09F8638B74000BDC09F8601B74087
S123C04000BDC09F860FB74000BDC09F8606B740008640BDC09FB74000C608CEC021A60099
S123C06008BDC0855A26F78601BDC09FB74000CEC000BDC08E86C0BDC09FB74000CEC01110
S123C080BDC08E20FE7D40002BFBB7400139A600084D2601397D40002BFBB7400120EF7D9D
S108C0A040002BFB39F8
S123FFD6C029C029C029C029C029C029C029C029C029C029C029C029C029C029C029C02977
S10DFFF6C029C029C029C029C02970
S9030000FC
